:020000020000FC
:080000000C94CE010C94CC001D
:040014000C944B01FC
:040034000C948A019D
:040040000C94F80024
:040048000C94610CA7
:100050000C94300CBF93AF93A8E8B1E016E02D915B
:100060003D91232B31F016961A95C9F7EF91FF9128
:1000700016C0ED93FD93ED920D93EF91FF910191D9
:100080000D9301910D9318973297ED93FC93E831FE
:1000900029F4F13019F40BA100640BA31197089512
:1000A0000A2F0B2B89F0ED91FD9114960D911D9166
:1000B00001931193EA3131F4F13021F40BA10F7B5C
:1000C0000BA3C3D7189701D00895FD92FD92FD921E
:1000D000FD92FD92FD92FD92FD92089507E0A8E841
:1000E000B1E0F3DF0A95E9F70895A8E8B1E026E06A
:1000F000BF93AF930D911D91012B21F012972F9378
:1001000009952F91AF91BF9118962A9589F7089577
:100110000D911D9112962D913C913F3F19F03A950A
:100120003C9389F0322F319533953E93222321F071
:10013000D801FD92FD920DC012972D913D91D801ED
:100140002D933D9306C01597FF93EF93A9DFEF9191
:10015000FF9108954A2F4B2B59F04D914E1741F4C2
:100160004D914F1729F40D931D9312960D931D93E6
:100170000895E8E8F0E0B9DF08955A9A0E94D70C94
:1001800002E01E8510FD03E00093690001D0089590
:10019000E89A0895E89808950F930FB70F93946025
:1001A0000F910FBF0F9118950F93F4BC05E005BD9B
:1001B0000F910895BF93AF93ADE7B0E0AF8FB8A3B1
:1001C000AF91BF910895FF8EF8A208950F93FF8E0F
:1001D000F8A201E005BB01E806BD01E000936E0056
:1001E0000F9108950F9300E000936E000F91089512
:1001F0000F9301E806BD78940FB70F931F93BF9339
:10020000AF93AF8DB8A10A2F0B2B51F01197AF8F81
:10021000B8A331F400910402002311F49860FCA209
:100220000DA1000F1E2D4F9B1127012B0DA3003890
:1002300049F40CA10E15A1F00BA108600BA3ECA2D0
:10024000B9DF0EC00F3721F00F3F51F413D008C0B3
:100250000CA1002329F09062FCA20BA1077F0BA345
:10026000AF91BF911F910F910FBF0F9118950CD0B7
:10027000ADDF0895B7DF01D0089510E810936D0049
:1002800014E010936800089510E010936D0010E0E2
:100290001093680008950F930FB71F930F93E7DF34
:1002A0000F911F910FBF0F91189504E000938100EB
:1002B0000AEF009385000AEE0093840022D008958F
:1002C000BF93AF93A8E0B7E0F894A9A3BAA378943A
:1002D000AF91BF910895BF93AF93A8E7B0E0F894B2
:1002E000A9A3BAA37894AF91BF910895F9A2FAA2F5
:1002F00008951F9309A11AA1012B09F00E2D1F913A
:10030000089501E000936F00F1DF089500E000938D
:100310006F0008950F930AEE009384000AEF009394
:10032000850078940FB71F930F93BF93AF93A9A144
:10033000BAA10A2F0B2B21F01197A9A3BAA301F49C
:100340000F81002329F00A9511F4906808850F8326
:1003500008890A9511F490640FE0088BAF91BF9162
:100360000F911F910FBF0F911895A89504B7077FA4
:1003700004BF0091600008610093600000270093B3
:1003800060000895F894A8950091600008610093BA
:1003900060000AE00093600078940895F894E5DF27
:1003A0002227E0E0F1E014E0002721930A95E9F725
:1003B0001A95D1F7C0ECD1E0FF24EE24E3949927FD
:1003C000882499240FEF0DA308AB02E30EA30FE4DA
:1003D0000FA3ECE1FBE1E0930001F0930101ECEAF3
:1003E000FCE1E0930102F0930202E0930401F09338
:1003F0000501EEE9FAE2E0933401F09335010AE4F5
:100400000093360106E019E4EFE1F1E01083349641
:100410000A95E1F7E0E9FEE1E0933C01F0933D014C
:10042000E8E6FFE1E0934001F0934101E2EBFFE1F8
:10043000E0934401F0934501EEEEFFE1E0934801C3
:10044000F0934901EAE5F0E2E0935001F0935101A5
:10045000E6E6F1E2E0935801F0935901E0E2F2E2BE
:10046000E0936001F0936101ECE8F2E2E09368014F
:10047000F0936901E4E3F3E2E0937001F09371011A
:10048000E4EBF3E2E0937801F0937901E2E8F4E23F
:10049000E0938001F09381010CE308830EE30F8366
:1004A00008870FE0088BE3EFF2E0EEAFFFAF01EC5F
:1004B0000093640079DEF9DE2ED10E940F0D0E94B8
:1004C000150C5BD563D5D9DE09DE01D60E87BDD507
:1004D000F2D50D8705E00A8BF98AF0D50B8F002342
:1004E00011F00FEF098BF0D50F87F4D5098F0E941B
:1004F000020D00910302002331F40E94CA0B0F3F4A
:1005000011F40E94B50AD4D50E8F002321F0F09289
:100510000401F0920501D5D50C87002311F40FE0FA
:1005200001C007E00A87098798D73DD279807BD040
:10053000B0D709810715D9F30A950983C1D11DDE0A
:10054000789417D60E94C30A14D60E942A0C6BD046
:1005500095FF19C09F7DE9E1F3E0EEAFFFAFE9D46D
:1005600000E5E4D3A0E4B1E0D7D360D05ED30FA11F
:100570000F3429F0BEDE0023C1F70FE4D7D3E3EF39
:10058000F2E0EEAFFFAF93FF23C004DE1BD50E9465
:10059000ED0C0C85002349F403E3B2D3A0E3B1E0F2
:1005A0009BD3ACE2B1E09CD305C006E3A9D3A0E1A4
:1005B000B1E092D338D0BCD20EA1023329F099DE3B
:1005C0000023C1F797D325D30E94F40CE1DDFCD4BE
:1005D00090FDE7D5BCCFFF93EF93EEADFFAD09954E
:1005E000EF91FF9108950F921F920F931F932F93F6
:1005F0003F934F936F938F93BF93AF93FF93EF937B
:100600005F937F9310D07F915F91EF91FF91AF91B6
:10061000BF918F916F914F913F912F911F910F91AA
:100620001F900F900895BAD024D00895E2D021D021
:1006300008950F921F920F931F932F933F934F9301
:100640006F938F93BF93AF93FF93EF935F937F93DA
:10065000EDDF7F915F91EF91FF91AF91BF918F910E
:100660006F914F913F912F911F910F911F900F907C
:10067000089592FF1EC01F8108850F83011B19F08A
:100680000E3108F406C00D8D002311F419D101C0FC
:1006900057D11091040210FF05C011FFA9D412FD1B
:1006A000AED406C0AEA5BFA50A2F0B2B09F0A0D46F
:1006B0009B7F97FF08C08BD40D8D002311F400D1D0
:1006C00001C03ED19F7796FF02C053DD9F7B94FF10
:1006D00021C00A890A9511F492D405E00A8B098D8C
:1006E000002311F001E03CD69F7E0BA101FF12C058
:1006F000198D0D8510230B8D102349F00B810430CB
:1007000031F4A4E1B1E0E6E3FDE100EFA3DC0BA1ED
:100710000D7F0BA30895209A219A229A239A389A42
:10072000399A3A9A3B9A539A549A559A5D9A5C9A96
:10073000089538B1307F0895582F580D5B0D5B98A0
:10074000052F5F70532B58B9029505B9562F590DD7
:100750005C0D052F5F70532B02955C985C9A5B9A39
:1007600058B905B95C985C9A0895562F580D5B0DE1
:100770005B98052F5F70532B58B9029505B9582F18
:10078000590D5C0D052F5F70532B02955C985C9A98
:100790005B9A58B905B95C985C9A08951127A0E056
:1007A000B1E0A10FBF1DA10FBF1DA10FBF1DA10F64
:1007B000BF1DED91FD91BD90CD90139509850395D9
:1007C00010170CF014C00E2F0F2B49F35D9A859172
:1007D0008823C9F3659145914423A9F34F3FF9F26A
:1007E00025912F934F932ED08F916F91F4CF5D9AD7
:1007F00008951127ACE3B1E0A10FBF1DA10FBF1DEC
:10080000A10FBF1DA10FBF1DED91FD91BD90CD901A
:10081000139514310CF014C00E2F0F2B59F35D9A61
:1008200085918823C9F3659145914423A9F34F3FEE
:1008300009F325912F934F9305D08F916F91F4CFAA
:100840005D9A089576DFDF01ECE9F3E0522F561B45
:100850000AF45195042F081B0AF40195051744F476
:10086000E5EBF3E0862768278627422724274227DF
:10087000481730F4842748278427622726276227D1
:10088000442E481A522E561A0AF451942224332424
:100890006624621710F4639401C06A94481770F0DC
:1008A0000995250C3F1C722D720D74153F041CF028
:1008B000660D24183F088395481790F7FD010895A9
:1008C0000F921F921F930F932F933F93FF93EF93DA
:1008D00057D31981139519831C3341F00A8D0023D6
:1008E00011F0FA8E23C069D0B1D021C090611E856D
:1008F000112321F4D9D50ED1B0D518C0F9821A81AF
:1009000013951A831C336CF01BA112601BA3FA828F
:100910001B8113951B83FED01B81183114F0FB82C1
:1009200005C01C8D112311F4DCD597D53DD0EF9176
:10093000FF913F912F910F911F911F900F9008955C
:100940001E85112339F11CD308850F8319811A954F
:1009500019831F3F41F00A8D002311F0FA8E19C050
:100960002CD074D017C01BE3198390611A811A959B
:100970001A831F3F71F41BE31A831BA112601BA390
:100980001B811A951B83C6D01B811F3F11F417E1F1
:100990001B830AD008951C8D0D8D102B19F484D55E
:1009A00003D00895089580D5B5D003D03AD098D01B
:1009B000089503D010D01DD00895EAE3F5E209812F
:1009C00015E0019FE00DF11D8F01E8E0F1E00083EB
:1009D00011839BD10895E6E6F6E20A8119E0019FB2
:1009E000E00DF11D8F01ECE0F1E0008311838DD16A
:1009F0000895E2E8F8E20A811CE0DFD60F930B814C
:100A0000DCD6022F25E0029F1F91100D29E0129FD6
:100A1000E00DF11D8F01E0E1F1E00083118375D15C
:100A2000089514D029D03ED00895000FE00FFF1D87
:100A300005911491000F111F0895EEEFFAE2F5DF12
:100A400008950F851EE300FD1AE408950981D8D6A4
:100A5000F4DFE0E2F1E00083118357D1F2DF185BAD
:100A60001283022FEADFECE1F1E0008311834DD124
:100A7000E8DF1C5A128308950A81C2D6DEDFE8E25D
:100A8000F1E00083118341D1DCDF185D1283022F76
:100A9000D4DFE4E2F1E00083118337D1D2DF1C5CC4
:100AA000128308950B810F8400FC05C0ECEEFBE27D
:100AB000E00FFF1D0491A4D6C0DFE0E3F1E0008366
:100AC000118323D1BEDF195F1283022FB6DFECE260
:100AD000F1E00083118319D1B4DF1C5E1283089505
:100AE0000F85002369F4EAECFAE20B810C3014F074
:100AF000E2EEFAE2E0933801F09339010EE305C02B
:100B0000F0923801F09239010AE400933A0100931F
:100B100036010895ECEAFCE1E0930102F093020251
:100B20000E8D002321F4E0930401F0930501089554
:100B30000EA1033389F495FF03C09F7D84D474C054
:100B400093FF72C004E3DCD0D5D0A8E2B1E0C4D0FA
:100B5000A4E2B1E0C5D068C0043389F495FF03C0B6
:100B60009F7D67D461C093FF5FC005E3C9D0C2D049
:100B7000A0E2B1E0B1D0ACE1B1E0B2D055C00533F4
:100B800059F495FF03C09F7D4AD44EC093FF4CC0DB
:100B900009E3B6D0AFD029C0063369F495FF03C08E
:100BA0009F7D51D441C093FF3FC007E3A9D0ACE083
:100BB000B1E092D039C0073369F495FF03C09F7D3F
:100BC00038D432C093FF30C008E39AD0A8E0B1E037
:100BD00083D02AC0083399F495FF03C09F7D1FD4AA
:100BE00023C093FF21C009E38BD0ACEDBDE1A093FE
:100BF0001401B0931501A4E1B1E06ED015C0093322
:100C000009F007C095FF03C09F7D6BD404C093FF1C
:100C10000BC04AD4C9DE68D0A0E0B0E0A0931401B4
:100C2000B093150102E36CD00895EEE8FCE00FA14B
:100C30000055102F110F110F000F010FE00FFF1DB6
:100C400095FF0AC09F7D05911591F80109950DAD9D
:100C500003950DAF35DB1AC093FF18C0329605918E
:100C60001591FF93EF93F8010DAD002309F009955D
:100C70000FA103950A350CF00FE458D0EF91FF91C6
:100C8000A591B5910A2F0B2B09F046D00895C2010A
:100C900000004401471865064C01EB06FF065401AD
:100CA000B906CF065C0107071B076401210735075A
:100CB0006C013D0751077401A006B2067C0159077B
:100CC000710784017907910700000895ED91FD9166
:100CD00012970FEFBFD90895F9DFA8A7B9A7089514
:100CE000F5DFAAA7BBA70895A8A5B9A5D9D9F8A6E5
:100CF000F9A60895AAA5BBA5D3D9FAA6FBA608957F
:100D0000977F0EA3F1DFDCDA0895A8A5B9A522DA52
:100D1000AAA5BBA51FDA0895D9DFACA7BDA7089582
:100D2000ACA5BDA5BDD9FCA6FDA60895977F0FA3D0
:100D3000FDAEC6DAF5DF0895ACA5BDA50BDA0895C2
:100D40000AAD019503950AAF01D008950AADE0E61A
:100D5000FDE06BDEE4E7F1E000831183EDDF089551
:100D6000B311C8110AAD1E8D19F0FBD409E50FA30C
:100D700008950EA9039507310CF004E10EAB01D0E4
:100D800008950EA90451E8E9FDE04FDEE4E5F1E045
:100D900000831183D1DF089561107E109D100EA98C
:100DA000109100020117B1F0163169F47ED40EA93A
:100DB0001F85112321F0053159F09BD409C004315E
:100DC00039F097D405C0063111F46FD401C091D425
:100DD00009E50FA308950DA9019503950DAB01D069
:100DE00008950DA9002319F40EE210E202C002E1F9
:100DF00010E2ECE4F1E0008311839EDF08950DA979
:100E00001B85011719F0DAD309E50FA308950FA97F
:100E1000019503950FAB01D008950FA9002319F494
:100E200004EC11E202C006EF11E2ECE5F1E0008310
:100E3000118382DF08950E851FA9011709F018D4C8
:100E4000089508AD0195039508AF01D0089508AD48
:100E5000002319F000E612E202C004E412E2E4E624
:100E6000F1E00083118368DF089508AD1D85011747
:100E700019F02FD409E50FA3089509AD0195039545
:100E800009AF01D0089509AD002319F008E013E27D
:100E900002C00CEE12E2ECE6F1E0008311834CDFBD
:100EA000089509AD1B8D011719F038D409E50FA37A
:100EB00008950E850E1108950BAD019503950BAFA6
:100EC00001D008950BAD002319F006E414E202C02E
:100ED00008E014E2ECE7F1E0008311832DDF0895D0
:100EE00008950BAD1C8D011719F099D309E50FA3D7
:100EF00008950E850E1108950CAD019503950CAF64
:100F000001D008950CAD002319F004EF14E202C0E3
:100F100006EB14E2E4E8F1E0008311830DDF0895AD
:100F200008950CAD1D8D011719F091D309E50FA39C
:100F300008950B850DAB55DF0C85002311F016E1EC
:100F400005C014E10F85002309F015E11EAB1093D5
:100F5000000217DF0E850FAB60DF0D8508AF77DF6E
:100F60000B8D09AF90DF0E8D0AAFF0DE0C8D0BAF4D
:100F7000A9DF0D8D0CAFC6DF0895569A5E980895CF
:100F80000D8500FF4E9A08955E98089557985F9AD0
:100F9000089508A90F3F71F4E8AAA9A9BAA90A2FD0
:100FA0000B2B41F4A8E1B1E0E6E7FDE100EF52D8F8
:100FB000A9ABBAAB08950FEF08ABA9A9BAA970D82D
:100FC000F9AAFAAAFF82089508850F8308950C8D67
:100FD00000FD0895AEA5BFA50A2F0B2B41F4A8E193
:100FE000B1E0E0E9FDE10FEF35D8AEA7BFA7089566
:100FF000AEA5BFA555D8FEA6FFA627D0089509899E
:101000000F3F71F0FF93EF93E4E0FCE2039507706C
:10101000098B000FE00FFF1D85909490EF91FF91D9
:101020000895ABA9BCA90A2F0B2B41F4A0E0B1E0B5
:10103000ECE1FBE100E50ED8ABABBCAB0895ABA98E
:10104000BCA92ED8FBAAFCAA08950BA106FD0EC0D0
:101050000E85002329F4F0921801F092190106C0C0
:10106000EAE6FDE1E0931801F09319010895A7E085
:10107000B0E016C0A0E0B0E013C0A6E0B0E010C041
:10108000A3E0B0E00DC0A2E0B0E00AC0A4E0B0E090
:1010900007C0A1E0B0E004C0A5E0B0E001E000C0FE
:1010A00000900402002019F400BD16E078D30895E2
:1010B000A7E0B0E012C0A0E0B0E00FC0A6E0B0E052
:1010C0000CC0A3E0B0E009C0A4E0B0E006C0A2E01C
:1010D000B0E003C0A1E0B0E000C011E060D30F3F7A
:1010E00009F4002708950F9309818EE1080F0C334E
:1010F0000CF00C5356D4882329F46DDA8981081733
:1011000029F0F8CF0CD48AD30F91089588E50F9178
:1011100008958F934AD4882311F45DDAFBCF8F9121
:10112000F5D3089542D4882311F455DAFBCF12D4B5
:1011300008958F933AD4882311F44DDAFBCF8F9121
:1011400018D0089532D4882311F445DAFBCF12D495
:1011500008950F932AD4882311F43DDAFBCF0F9121
:10116000002319F0E8EFFDE2F5C3ECEFFDE2F2C376
:101170000895E4EFFDE2EEC3AED895FF02C09F7D77
:1011800001D929DAB6D80023C1F70895F5DFF4DFD5
:101190000895C8DFCEDFF0DF0895C4DFCADFF6DFD1
:1011A00008958F931F930F932F933F93BF93AF9304
:1011B000FF93EF930F921F92B2D330D3883509F08B
:1011C0008EC0EAE3FCE2AEDF8EDFA3DFB2DF843560
:1011D00009F43AC0843409F46AC0833509F465C05F
:1011E0008C3411F476D27BC0813411F441D277C0B3
:1011F000863511F4ACD273C0833411F4DFD16FC0E3
:101200008E3411F452D26BC0803511F472D267C0A3
:10121000823411F483D263C0813511F400D25FC0EF
:10122000823511F414D25BC0863411F49AD257C0BF
:10123000883411F4BED253C08D3419F40E941F1BA0
:101240004EC0883571F1BDCFE4E6FCE26BDF55D0CE
:1012500038F16DD15FDC6DDFECE7FCE263DF4DD090
:10126000F8F05DD166DFE4E9FCE25CDF46D0C0F077
:101270000E85002351F48F9389818F938FDA8F919C
:1012800008D109810817C9F38F913FD1EA8E0981EE
:101290000A95098315DB9B774CDF002761D004C0DA
:1012A00082DBE6EBFDE23EDF1AC06DD118C0ECEA4E
:1012B000FCE238DF22D0A8F352D13BDFE4ECFCE2C1
:1012C00031DF1BD070F343D134DFECEDFCE22ADFD9
:1012D00014D038F334D12DDF002742D000C029DFED
:1012E000EA8E1F900F90AF91BF91EF91FF913F91C8
:1012F0002F910F911F918F910895F5DE0ADF8835A8
:1013000011F4089408950DD0C0F3082FECDE01DF2E
:101310008835B9F306D0D0F31AE0019F800D889488
:101320000895803328F08A3318F480538894089500
:1013300008940895E4E1FCE2F5DE82E3EADE8EE261
:10134000E8DE86E3E6DEF5DE089552D28F938295DD
:101350008F705AD28D938F918F7056D28D9308953E
:1013600024D3882311F437D9FBCFFF93EF93BF9396
:10137000AF930F93A5E0B2E011D080E28D9329D016
:101380000F91002321F08DE08D938AE08D93FD92E3
:10139000F1D2AF91BF91EF91FF9108958C81D5DF8C
:1013A0008DE28D938D81E0E0FEE28A95880F880FB3
:1013B000E80FFF1D85918D9385918D9385918D9378
:1013C0008DE28D9382E38D9380E38D938E81BDDFDB
:1013D00008958B81BADF8AE38D938A81B6DF8AE331
:1013E0008D938981B2DF0895E0D2882311F4F3D878
:1013F000B7CFFF93EF93BF93AF930F93A5E0B2E006
:10140000E8DF0F91002321F08DE08D938AE08D932A
:10141000FD92B0D2AF91BF91EF91FF9108950981F4
:1014200003950C3308F0002709830E946001BCDAA1
:1014300008950A8103950C3308F000270A830E945F
:101440006001B2DA08950B810395083108F0002796
:101450000B830E946001A8DA08950F938F9315E023
:10146000E3D28F73B5D180320CF08E2D8C8317E0D0
:10147000DBD28F71ADD18D300CF08E2D8D8318E0C5
:10148000D3D2A6D183360CF088278E838F910F910B
:1014900008958F9312E0C8D28F779AD18C330CF0D5
:1014A000882789838F9108958F9312E0BDD287FD9D
:1014B00070DD8F778DD18C330CF08827898313E012
:1014C000B3D28F7785D18C330CF088278A8314E0D0
:1014D000ABD28F737DD188310CF088278B838F91AD
:1014E000089580910402882379F4898181D112E0E2
:1014F000082FBCD28A817CD113E0082FB7D28B8110
:1015000077D114E0082FB2D208958F93082F0C33AF
:1015100020F489836DD112E0A9D28F910895082F0C
:101520000C3320F48A8364D113E0A0D20895082FED
:10153000083120F48B835CD114E098D20895082FF1
:10154000003220F48C8354D115E090D20895082FF6
:101550000C3020F48D834CD117E088D20895082FE9
:101560008E8346D118E082D208958827CEDF88275F
:10157000D6DF8827DCDF81E0E2DF81E0E8DF882753
:10158000EEDF8ADD0895D6DE0027EADE80E2C1DDE7
:1015900082E50E85002309F081E4BBDD0D85002383
:1015A00011F48CE4B6DD0B8D002311F482E4B1DD7F
:1015B000098D002311F086E5ACDD08952F93E4EF4B
:1015C000FCE2B0DD0B85002339F01CD20027222776
:1015D0001A85ECE1FBE109C015D010D20E2D2FEFDA
:1015E0008824992411E0E0E2F5E21987E0930001F4
:1015F000F09301011B8D112309F4298B0B87A9DDC1
:101600002F9108950C8D002321F01EE318871F836E
:10161000FC8E0D8D002309F0FD8EBDD908950E8539
:1016200000FD04C0E4E7FDE27DDD10C0EAE5FDE277
:1016300079DD0C8D002319F01EE3002702C012E0B3
:101640000E2D18871F830C8F84DDA5D908950E8574
:1016500000FD04C0E4E7FDE265DD09C0E6E6FDE269
:1016600061DD0D8D019503950D8F73DD94D908957E
:10167000E4E3FDE257DD0E85002339F0C3DF0027E8
:10168000F0921801F092190107C00395EAE6FDE116
:10169000E0931801F09319010E87F5DC5ADD0091F3
:1016A000040200FF0E94C2010895EAE0FDE23ADD73
:1016B0000C85002319F000271FE002C0039517E0F6
:1016C0000C8719871A87DCDC0195039542DD22DA45
:1016D0000895ECE1FDE226DD0D85002311F00027E1
:1016E00002C0039551DC0D87C5DC0195039531DD02
:1016F0000895ECE2FDE216DD0F85019503950F8755
:10170000C5DC1EE300FD1AE40195039522DD2F2DB3
:1017100003D0E6D986D9089584D90895E6E4FDE298
:1017200001DD0B8D019503950B8F0F93A6DC0195C1
:1017300003950FDD0F911B85112341F4002329F040
:101740000FEF098B8824992401C0F98A0895E2E2F9
:10175000FDE2E8DC098D01950395098F9ADCF9DC3F
:101760000895E2EAFDE2DEDC0E8D002331F0002771
:10177000E0910102F091020203C00395E0E0F0E085
:10178000E0930401F09305010E8F71DC0195039540
:10179000E0DC0895A5E0B0E011E001D00895A1BD1E
:1017A000B2BD119611FDFA9A1FBBF999FECF00B593
:1017B0000895E0E3FEE2B6DC0895222738E0000F4A
:1017C000221F211710F00395211B3A95C1F70895A8
:1017D0000F921F920F938F9382958F700AE0809FD4
:1017E000002D8F918F70800F0F911F900F90089593
:1017F000082F1AE0E2DF07700295022B802F089570
:101800001AE0DBDF07700895FF93EF93ECEDFBE246
:10181000E80FFF1D8491EF91FF910895813624F028
:101820008B3710F400E2801B089510E41093C4007D
:10183000F092C500F092C00018E41093C10016E0C9
:101840001093C200EB8AFF8AF88EFC8AFD8A1FEF94
:101850001E8B08951091C10010691093C100089566
:101860000F930FB70F931F93FF93EF930E890F3FC3
:1018700079F00395E5E0F2E0E00FFF1D1081112300
:1018800019F40FEFEB8A02C01093C6000E8B12C042
:10189000EC89FD890E2F0F2B39F0EF5FFF4F14916C
:1018A000112321F4FC8AFD8AEB8A04C01093C60040
:1018B000EC8BFD8BEF91FF911F910F910FBF0F915B
:1018C00018950F930FB70F930BA102FD0C947E1B7D
:1018D0001F932F933F93FF93EF932091C6000F899F
:1018E000302F03950F70188D011739F00F8BE5E835
:1018F000F2E0E30FFF1D20839160EF91FF913F9194
:101900002F911F910F910FBF0F9118950F930B8976
:101910000023E9F3FB8A8093C6000F91089590FF9E
:10192000FECF0F931F93FF93EF931F89088D882796
:10193000011751F0E5E8F2E0E00FFF1D808103950B
:101940000F70088F011709F49E7FEF91FF911F918F
:101950000F9108950F93FF93EF930B890023E9F301
:10196000FB8AEC8BFD8B04910093C600EF91FF91F5
:101970000F9108950F93FF93EF930B890023E9F3E1
:10198000FB8AFE8AE5E0F2E00081002321F40FEFFC
:101990000E8BEB8A02C00093C600EF91FF910F916E
:1019A0000895882790FD839508958B8908951F9346
:1019B0000F9328D01FE000E459D01EE001E856D074
:1019C00011E001E153D00F911F9108951FE000E451
:1019D0004DD011E001E14AD008951EE000E846D064
:1019E00011E000E143D008951FE000E43FD01EE085
:1019F00001E83CD011E001E139D008951DE000E894
:101A000035D008951DE0002731D008950000000072
:101A100000000000000000000000000008953C9A53
:101A20003D9A449A459A08953F9333273A9519F47D
:101A3000E092030217C0B1F067D0E8DF02EA3FD0BE
:101A4000E5DF33D098F3012F3AD0E0DF2ED070F3EA
:101A500055D05AD003EA33D0D9DF27D038F33CD061
:101A6000449A459A4BD0802F3F9108953F93332756
:101A70003A9519F4E092030215C046D0C7DF0F93E0
:101A800002EA1DD0C3DF11D00F9190F30F93012F05
:101A900016D00BD00F9160F30F9311D006D00F9199
:101AA00038F300002BD03F9108953C98449A089455
:101AB000459AACDF349B889445983C9A08953F93AF
:101AC00038E0449A000F08F04498459A9FDF459803
:101AD0003A95B9F73F9108953F933C98449A00E0B6
:101AE00038E0459A089492DF349B8894001F45980B
:101AF0008DDF3A95B1F73C9A3F9108954498459A05
:101B000000000000449A0895449A459A000000009D
:101B10004498000000004598000008957AEB7AD9B7
:101B20000080E883EB89EB8CE88CE580D98CD900C8
:101B3000862483277D277A247A187D1583158618B5
:101B4000861B831E7D1E7A1B00E086E389E989ECF3
:101B500086EC83E980EC7DEC7AE977E377E07A0044
:101B6000E380E980001F831C801C80168013831390
:101B70008616891C891F861F7A1C771677137A00B0
:101B800080FE80F2008DFE8CF9009AFC99F700A689
:101B9000F8A5F400B3F4B1EF00BFEEBAE500CAE671
:101BA000C7E200D4DED0DA00DDD5D9D100E5CBE143
:101BB000C800EDBFE4BA00F3B4EEB200F7A7F3A695
:101BC00000FB9BF69A00FD8EF88D00FD80F18000F1
:101BD000FD73F87400FB66F66700F75AF35B00F3D9
:101BE0004DEE4F00ED41E44600E536E13900DD2CD5
:101BF000D93000D423D02700CA1BC71F00BF13BA97
:101C00001C00B30DB11200A609A50D009A05990A92
:101C1000008D038C08007F037F0F007203730800A0
:101C20006505660A0059095A0D004C0D4E12004117
:101C300013461C00351B381F002B232F2700222C96
:101C40002630001A361E390012421B47000C4D1177
:101C50004F00085A0C5B00046609670002730774A2
:101C60000002810E8100028E078D00049B099A00FC
:101C700008A70CA6000CB411B20012BF1BBA001AC0
:101C8000CB1EC80022D526D1002BDE2FDA0035E688
:101C900038E20040EE45E5004CF44EEF0059F85AAA
:101CA000F40065FC66F70072FE73F9FFB5E4B5D287
:101CB0000000D2BBD5BEDBBEDEBBDEB8D2ACDEAC34
:101CC0000000E04CD44CDD55DD430000B831AC31B0
:101CD000AC28B528B825B822B51FAF1FAC2200002C
:101CE00047315331532E502B4D254D1F0000224CB0
:101CF0001F4F1F52225528552B522B4F284C224C38
:101D00001F491F46224328432B462B49284C0000DD
:101D100021BE21AC000027BB2ABE30BE33BB33AF8F
:101D200030AC2AAC27AF27BB000049E449D2000001
:101D300053E453D2FF00B2A4B2A6BAA6BA9AB29A9A
:101D4000B29C00BE9ABE9EC49EC49ABE9A00C49A1B
:101D5000C4A600C79AC7A6CDA6CFA4CFA2CDA0C7C0
:101D6000A000CDA0CF9ECF9AFF007CBA80C684BAD7
:101D70000082BE7EBEFF7CBA7CC682C684C484C29A
:101D800082C07CC082C084BE84BC82BA7CBAFF00A0
:101D90007CBA7CC682C684C484C282C07CC0FF0078
:101DA000A999AC99AD98AD94AC93A993A99900B9B0
:101DB00099B599B593B99300B896B59600C093C0FC
:101DC00099C297C499C49300CB98CC99CE99CF98D7
:101DD000CF94CE93CC93CB94CB98FF003A933A997F
:101DE0003D993E983E973D963A96004699469447CF
:101DF0009349934A94004A994A93005698559953A7
:101E00009952985297539655965695569455935382
:101E1000935294005E995E93005E96629600629380
:101E200062990076997A99007899789300829883DC
:101E30009985998698869485938393829482980055
:101E40009E989D999B999A989A979B969D969E95F8
:101E50009E949D939B939A9400A699AA9900A89901
:101E6000A89300B293B499B69300B595B39500BE0C
:101E700093BE99C199C298C297C196BE9600C19669
:101E8000C295C29300CA99CE9900CC99CC93FF0019
:101E900029EC2FEC31EA31E22FE029E029EC003582
:101EA000EC35E237E03BE03DE2003DEC3DE0004157
:101EB000EC49EC0045EC45E00055EA53EC4FEC4DA5
:101EC000EA4DE24FE053E055E20059EC59E0005989
:101ED000E661E60061E061EC0065EC6DEC0069EC48
:101EE00069E00071E071EC77EC79EA79E877E67106
:101EF000E60077E679E479E0007DEA7FEC83EC8523
:101F0000EA85E283E07FE07DE27DEA0089E089EC1A
:101F100091E091EC0097E09BE00099E099EC00974C
:101F2000EC9BEC00A1ECA9E000A9ECA1E000B9EC6D
:101F3000BDE0C1EC00C5EAC7ECCBECCDEACDE8C50D
:101F4000E0CDE000D3E0D3E4D7E4D7E0D3E000E590
:101F5000EAE3ECDFECDDEADDE2DFE0E3E0E5E2E549
:101F6000E4E3E6DFE6DDE4FF29C229CE2FCE31CC63
:101F700031CA2FC829C82FC831C631C42FC229C2BF
:101F80000035CC37CE3BCE3DCC3DC43BC237C2350D
:101F9000C435CC0041CC43CE47CE49CC49C447C21E
:101FA00043C241C441CC004DCE55CE0051CE51C2AA
:101FB000FF0029BA2FBA31B831B02FAE29AE29BAF5
:101FC000003DBA35BA35AE3DAE003BB435B4004144
:101FD000AE41BA45B649BA49AE004DB84FBA53BA48
:101FE00055B855B053AE4FAE4DB04DB8FF0031A40B
:101FF0002FA62BA629A4299C2B9A2F9A319C003519
:102000009A39A63D9A003B9E379E0041A6419A49C7
:102010009AFF59A45BA65FA661A4619C5F9A5B9A34
:10202000599C59A400659A65A66D9A6DA6FF59A49E
:102030005BA65FA661A4619C5F9A5B9A599C59A4B8
:10204000006DA665A6659A0065A06BA00079A671D3
:10205000A6719A0071A077A0FF0029862992318687
:102060003192003592358837863B863D88003D9217
:102070003D860041864192458E499249860055929F
:102080004D924D86558600538C4D8C005986599241
:102090005F926190618E5F8C598C005F8C618A6168
:1020A000860067866B8600698669920067926B92EC
:1020B00000799077927392719071887386778679A0
:1020C00088FF8D928D8600959097929B929D909D12
:1020D0008E95869D8600A192A18600A18CA98C0078
:1020E000A986A99200AD86AD92B392B590B58EB394
:1020F0008CAD8C00B38CB58AB586FF0089908B922D
:102100008F929190918E89869186009D8C958C9B63
:10211000929B8600A192A18600A18CA98C00A98621
:10212000A99200AD86AD92B392B590B58EB38CAD49
:102130008C00B38CB58AB586FF0089908B928F9204
:10214000919091888F868B8689888990009D929541
:1021500092958600958C9B8C00A992A192A18600F5
:10216000A18CA78CFF002972297E2D7A317E3172D5
:10217000003572397E3D72003B76377600497C47E8
:102180007E437E417C417A4378477849764974475B
:102190007243724174004D7E557E00517E51720033
:1021A000617E597E59726172005F7859780065725C
:1021B000657E6B7E6D7C6D7A6B786578006B786D73
:1021C000766D72FF7D727D7E837E857C857A8378D5
:1021D0007D780083788576857200897E917E008D7A
:1021E0007E8D72009D7C9B7E977E957C9574977208
:1021F0009B729D74FF007D72817E85720083767F65
:102200007600897E8D72917E009572957E9B7E9D73
:102210007C9D7A9B789578009B789D769D72FF00D7
:10222000296A295E315E003D6A356A355E3D5E0091
:102230003B64356400416A476A49684960475E41CA
:102240005E416AFF59685B6A5F6A616861605F5EF0
:102250005B5E5960596800655E656A6D5E6D6AFF18
:1022600059685B6A5F6A616861605F5E5B5E596066
:102270005968006D6A656A655E0065646B64007923
:102280006A716A715E0071647764FF00294A295699
:102290002F56315431522F5029502F50314E314C3E
:1022A0002F4A294A003556354C374A3B4A3D4C00A7
:1022B0003D563D4A00414A415647564954495247C6
:1022C000504150004750494E494A004D4A4D5655DD
:1022D0004A5556005B4A5F4A005D4A5D56005B56B0
:1022E0005F5600654A65566D4A6D56FF7D547F56B0
:1022F00083568554854C834A7F4A7D4C7D540089A2
:102300004A8956914A9156FF7D547F56835685548B
:10231000854C834A7F4A7D4C7D540091568956896D
:102320004A0089508F50009D569556954A00955009
:102330009B50FF0029422F42314031382F36293639
:1023400029420037363B3600393639420037423BA6
:10235000420041364542493600473A433A004D4231
:102360004D365536FF006D426542653600653C6B63
:102370003C0071427138733677367938007942798A
:1023800036007D427D36853600894289369136FF9A
:1023900065366542693E6D426D36007336773600AC
:1023A000753675420073427742007D367D42853630
:1023B0008542FF00312C2F2E2B2E292C292A2B2849
:1023C0002F28312631242F222B2229240035223593
:1023D0002E3B2E3D2C3D2A3B28352800492E412EF0
:1023E00041224922004728412800552E4D2E4D22DA
:1023F00055220053284D2800592E5F2E612C612450
:102400005F225922592EFF007122712E7922792ED6
:10241000007D2C7F2E832E852C852483227F227D98
:10242000247D2C008922892E8F2E912C912A8F2891
:102430008928008F2891269122009522952E992A8D
:102440009D2E9D22FF00792E712E7122007128771A
:1024500028007D22812E85220083267F2600912C54
:102460008F2E8B2E892C892A8B288F2891269124B8
:102470008F228B22892400952E9D2E00992E992241
:10248000FF00291A2F1A311831102F0E290E291A80
:1024900000370E3B0E00390E391A00371A3B1A006E
:1024A000410E411A471A491849164714411400476A
:1024B000144912490EFF590E591A610E611A00652E
:1024C00018671A6B1A6D186D106B0E670E65106524
:1024D0001800710E711A771A791879167714711419
:1024E0000077147912790E007D0E7D1A8116851AF7
:1024F000850EFF00590E591A5F1A611861165F1494
:102500005914005F146112610E006D1A651A650E90
:102510006D0E006B14651400711A750E791AFF00A8
:1025200001FE0101FE01FEFE01FEFE010101FEFEB3
:1025300001FE0101FE01FEFEFF0080EC8080FF8BAA
:10254000EC8080FF96EA8080FFA1E78080FFABE30C
:102550008080FFB6DE8080FFBFD88080FFC8D1803A
:1025600080FFD0C98080FFD7C08080FFDDB680802B
:10257000FFE2AC8080FFE6A28080FFE9978080FFC9
:10258000EB8C8080FFEB808080FFEB758080FFE923
:102590006A8080FFE65F8080FFE2558080FFDD4A31
:1025A0008080FFD7418080FFD0388080FFC8308096
:1025B00080FFBF298080FFB6238080FFAB1E808014
:1025C000FFA11A8080FF96178080FF8B158080FF07
:1025D0007F158080FF74158080FF69178080FF5E03
:1025E0001A8080FF541E8080FF4A238080FF40298C
:1025F0008080FF37308080FF2F388080FF28418027
:1026000080FF224B8080FF1D558080FF195F8080F6
:10261000FF166A8080FF14758080FF14818080FF20
:10262000148C8080FF16978080FF19A28080FF1D88
:10263000AC8080FF22B68080FF28C08080FF2FC939
:102640008080FF37D18080FF40D88080FF49DE80C6
:1026500080FF54E38080FF5EE78080FF69EA80802E
:10266000FF74EC8080FF828080E67E808280FF8124
:10267000808AE67E818180FF818095E47E818180F1
:10268000FF81809FE27E818180FF8180A9DE7E8143
:102690008180FF817FB3D97E82817FFF817FBBD321
:1026A0007E82817FFF817FC4CC7E82817FFF817F9C
:1026B000CBC57E82817FFF817FD2BC7E82817FFFFE
:1026C000807FD8B37F82807FFF807FDDAA7F82807A
:1026D0007FFF807FE1A07F82807FFF807FE3967F06
:1026E00082807FFF807FE58B7F82807FFF7F7EE51A
:1026F0008080827F7EFF7F7FE57680827F7FFF7F85
:102700007FE36B80827F7FFF7F7FE16180827F7FBD
:10271000FF7F7FDD5780827F7FFF7E7FD84D818264
:102720007E7FFF7E7FD24581827E7FFF7E7FCB3C96
:1027300081827E7FFF7E7FC43581827E7FFF7E7FA8
:10274000BB2E81827E7FFF7E7FB32881827E7FFFCA
:102750007E80A92381817E80FF7E809F1F81817E74
:1027600080FF7E80951D81817E80FF7E808A1B8117
:10277000817E80FF7E817F1B82807E81FF7E8175CE
:102780001B81807E81FF7E816A1D81807E81FF7E2C
:1027900081601F81807E81FF7E81562381807E81C2
:1027A000FF7E814D2881807E81FF7E82442E817F45
:1027B0007E82FF7E823B35817F7E82FF7E82343C3B
:1027C000817F7E82FF7E822D45817F7E82FF7F8298
:1027D000274E807F7F82FF7F822257807F7F82FF0C
:1027E0007F821E61807F7F82FF7F821C6B807F7F64
:1027F00082FF7F821A76807F7F82FF80821A817FAC
:102800007E8082FF80821A8B7F7F8082FF80821C85
:10281000967F7F8082FF80821EA07F7F8082FF80E4
:102820008222AA7F7F8082FF808227B37F7F80827F
:10283000FF81822DBC7E7F8182FF818234C57E7FB5
:102840008182FF81823BCC7E7F8182FF818244D363
:102850007E7F8182FF81824CD97E7F8182FF818150
:1028600056DE7E808181FF818160E27E808181FFF2
:1028700081816AE47E808181FF818175E67E80812D
:1028800081FF828080BC7E808280FF818086BC7ECA
:10289000818180FF81808CBB7E818180FF818092DD
:1028A000BA7E818180FF818098B77E818180FF819F
:1028B0007F9EB47E82817FFF817FA3B17E82817FF4
:1028C000FF817FA8AD7E82817FFF817FACA97E8260
:1028D000817FFF817FB0A47E82817FFF807FB39E56
:1028E0007F82807FFF807FB6997F82807FFF807F9D
:1028F000B9937F82807FFF807FBA8D7F82807FFF48
:10290000807FBB877F82807FFF7F7EBB8080827FCE
:102910007EFF7F7FBB7A80827F7FFF7F7FBA74805C
:10292000827F7FFF7F7FB96E80827F7FFF7F7FB650
:102930006880827F7FFF7E7FB36281827E7FFF7EA1
:102940007FB05D81827E7FFF7E7FAC5881827E7FFB
:10295000FF7E7FA85481827E7FFF7E7FA35081828D
:102960007E7FFF7E7F9E4D81827E7FFF7E80984AA4
:1029700081817E80FF7E80924781817E80FF7E8084
:102980008C4681817E80FF7E80864581817E80FFAE
:102990007E817F4582807E81FF7E81794581807E38
:1029A00081FF7E81734681807E81FF7E816D4781BC
:1029B000807E81FF7E81674A81807E81FF7E816289
:1029C0004D81807E81FF7E825C50817F7E82FF7E92
:1029D000825754817F7E82FF7E825358817F7E8220
:1029E000FF7E824F5D817F7E82FF7F824C63807F8E
:1029F0007F82FF7F824968807F7F82FF7F82466E71
:102A0000807F7F82FF7F824574807F7F82FF7F820D
:102A1000447A807F7F82FF808244817F7E8082FF34
:102A2000808244877F7F8082FF8082458D7F7F8088
:102A300082FF808246937F7F8082FF808249997FD8
:102A40007F8082FF80824C9E7F7F8082FF81824FC9
:102A5000A47E7F8182FF818253A97E7F8182FF8154
:102A60008257AD7E7F8182FF81825CB17E7F8182D1
:102A7000FF818261B47E7F8182FF818167B77E8022
:102A80008181FF81816DBA7E808181FF818173BBED
:102A90007E808181FF818179BC7E808181FF24538A
:102AA000245526552653245300244F244D264D26C5
:102AB0004F244F0044534455465546534453004415
:102AC0004F444D464D464F444FFF644B68576C4B47
:102AD000006A4F664F00704B705774537857784BAD
:102AE000FF00644B64576A576C556C536A516451CC
:102AF0000000704B705774537857784BFF0089155E
:102B0000931596159E15AC15B115BB15C815CF15A7
:102B1000E015040C060E0A0E0C0C0C040A02060248
:102B20000404040CFF00080E0802FF00040C060E4B
:102B30000A0E0C0C0C0A04020C02FF00040C060E18
:102B40000A0E0C0C0C0A0A080C060C040A020602F7
:102B500004040006080A08FF0C0804080A0E0A020A
:102B6000FF000C0E040E04080A080C060C040A02EE
:102B700006020404FF000C0C0A0E060E040C0404EA
:102B800006020A020C040C060A0806080406FF00E6
:102B9000040E0C0E0C0C0A0A08060802FF000608B8
:102BA000040A040C060E0A0E0C0C0C0A0A0806088D
:102BB0000406040406020A020C040C060A08FF00BC
:102BC0000C0A0A080A080608040A040C060E0A0E73
:102BD0000C0C0C040A0206020404FF0030313233EC
:102BE0003435363738394142434445460C010203F7
:102BF0000405060708090A0B0C0102030405060771
:102C000008090A0B0000010001010001FF01FF009B
:102C1000FFFF00FF447574636874726F6E697820FB
:102C2000415652204F7363696C6C6F73636F7065AC
:102C300020436C6F636B20560000456E74657220F4
:102C4000636F6D6D616E642028412C422C432C44CF
:102C50002C462C482C4C2C4E2C502C532C542C569F
:102C6000293A0000456E74657220322064696769F4
:102C70007420686F7572733A20202000456E746569
:102C8000722032206469676974206D696E7574659D
:102C9000733A2000456E746572203220646967695A
:102CA00074207365636F6E64733A2000456E7465BB
:102CB00072203220646967697420796561723A20F4
:102CC00020202000456E7465722032206469676997
:102CD00074206D6F6E74683A20202000456E746514
:102CE000722032206469676974206461793A202017
:102CF0002020200043616C6962726174696F6E20EC
:102D00005061747465726E2000004E756D65726955
:102D10006320646973706C61792000004C45442025
:102D20000000566572626F7365200000414D2F50A0
:102D30004D20000041565220436C6F636B204D6163
:102D40007374657220004275726E2D696E20507228
:102D50006576656E74696F6E200046617374204DF0
:102D60006F646520000052657665727365204D6F53
:102D700064652000526571756573746564206D6FBC
:102D800064652072657175697265732041565220C1
:102D9000636C6F636B204D6173746572204D6F645B
:102DA0006500416C6C2044696769747320646973C1
:102DB000706C6179200043616E63656C206F7220D6
:102DC00054696D656F7574004E6F7420456E74653F
:102DD00072696E672044656D6F204D6F64650000F9
:102DE000505053207369676E616C2069676E6F7213
:102DF000656400000D0A00004F6E00004F6666001B
:102E00004A616E1F4665621C4D61721F4170721EE1
:102E10004D61791F4A756E1E4A756C1F4175671F9B
:102E20005365701E4F63741F4E6F761E4465631F9B
:102E3000447574636874726F6E6978204F73636948
:102E40006C6C6F73636F706520436C6F636B2048AD
:102E5000656C703A0D0A413A20546F67676C6520C3
:102E60004D617374657220436C6F636B206265748F
:102E70007765656E2041565220616E64205254433E
:102E80000D0A423A20546F67676C65204275726E76
:102E90002D696E2070726576656E74696F6E0D0AAD
:102EA000433A20446973706C61792043616C6962B4
:102EB000726174696F6E207061747465726E0D0A50
:102EC000443A204368616E676520446174650D0A69
:102ED000463A20546F67676C6520416C6C204469EA
:102EE0006769747320446973706C61790D0A4C3A98
:102EF00020546F67676C65204C454420626C696E96
:102F00006B696E670D0A4E3A20546F67676C6520D7
:102F10004E756D6572696320446973706C617920C8
:102F20000D0A503A20546F67676C6520414D2F5051
:102F30004D200D0A533A20446973706C6179205317
:102F40007461747573200D0A543A204368616E678A
:102F5000652054696D650D0A563A20546F67676C99
:102F60006520566572626F7365204F757470757455
:102F70000D0A0000E0EAFDE1E0931401F093150171
:102F80000895E0E0F0E0E0931401F0931501089556
:102F90000C850023D9F50E94550B36C00C85002303
:102FA000A9F10E94550B30C00F85002379F50E94CE
:102FB000790B2AC00F85002349F10E94790B24C0A8
:102FC0000E8D002319F50E94B10B1EC00E8D00233B
:102FD000E9F00E94B10B18C00D850023B9F40E94DE
:102FE000690B12C00D85002389F00E94690B0CC08B
:102FF0000B85002361F00E94DE0A06C00B850023CA
:1030000031F40E94DE0A00C00E94990800C00895B1
:10301000098D0023E1F30E94A70BF6CF098D002351
:10302000B1F70E94A70BF0CF0E85002381F30E9419
:10303000380BEACF0E85002351F70E94380BE4CFFE
:103040000C8D002321F30E940F0BDECF0C8D00238B
:10305000F1F60E940F0BD8CF0D8D0023C1F20E9414
:10306000270BD2CF0D8D002391F60E94270BCCCFDA
:103070000895F98A08950E94F80708950E94E707C5
:1030800008950E94DB0708950E94C907089501E092
:10309000009304020E94BA17D3DFDEDFA9DFE3EF5B
:1030A000F2E0EEAFFFAFE8E4F2E30E94C908ECEE15
:1030B000F2E30E94C9080E94C8170E94E017EAE1E3
:1030C000F3E30E94C9080E94E617ECE3F3E30E94D1
:1030D000C9080E94D4170E94CE17EAE5F3E30E94C4
:1030E000C9080E94DA17ECE7F3E30E94C908EEE989
:1030F000F3E30E94C9080E94D4170E94BC080E94F2
:10310000E0170E94BC080E94DA170E94BC080E94C7
:10311000E6170E94C8170E94BC080E94E6170E948A
:10312000CE170E94BC080E94E0170E94C8170E9498
:10313000BC080E94E6170E94DA170E94CE170E9470
:10314000BC080E94EC17EAEBF3E30E94CD080E9452
:10315000F217E4EDF3E30E94CD080E94FE17E8EEBB
:10316000F3E30E94CD080E94F817E2E0F4E30E9426
:10317000CD080E941A18E4E1F4E30E94CD080E94F1
:103180002618E6E4F4E30E94CD080E94C6080E94D7
:103190002018E8E5F4E30E94CD080E943218ECE61E
:1031A000F4E30E94CD080E942618EEE7F4E30E94A3
:1031B000CD080E94C6080E94020B009304020E94E0
:1031C0004418ECEBF4E30E94CD080E94C60803E02B
:1031D000009304020E9441180E943E18EEE0F5E3BD
:1031E0000E94CD080E94C6080E943B180E94110848
:1031F000EEE5F5E30E94CD0805E0009304020E948D
:103200001F080E943918ECE7F5E30E94CD080E94E0
:10321000C608F09204020E943818E9E1F3E0EEAF2C
:10322000FFAFE8ECF2E30E94CD080E94C608E3EF8E
:10323000F2E0EEAFFFAFECEDF5E30E94C9080E94AB
:10324000C1170E94C2010895546869732064656DB6
:103250006F206D6F64652073686F777320736F6D77
:1032600065206F6620746865206361706162696CB7
:103270006974696573206F6620746865204475748D
:10328000636874726F6E69780D0A415652204F73ED
:1032900063696C6C6F73636F706520436C6F636BF5
:1032A0002E20497420707265736572766573207480
:1032B0006865207374617465206F6620796F75721C
:1032C00020636C6F636B2E004865726520796F75A3
:1032D0002063616E2073656520746865206F6E2DB4
:1032E00073637265656E206D656E75004865726505
:1032F0002061726520736F6D65206F66207468654C
:1033000020436C6F636B20446973706C6179732028
:10331000737570706F7274656400416E616C6F6775
:1033200020436C6F636B2077697468206D696E69E8
:103330006D616C206469676974730000416E616C33
:103340006F6720436C6F636B207769746820616CD2
:103350006C20646967697473000041646420746858
:103360006520323420686F757273206E756D6572DA
:10337000696320646973706C617900004F72206129
:1033800064642074686520414D2F504D206E756D2A
:103390006572696320646973706C617900004D69BE
:1033A0007820616E64204D617463682061732079B8
:1033B0006F7520706C65617365005475726E207452
:1033C0006865204C454420626C696E6B696E6720AD
:1033D0006F666600416E64207475726E2069742099
:1033E0006261636B206F6E005475726E206F6E2089
:1033F00043616C6962726174696F6E204D6F6465C0
:1034000000005475726E206974206261636B206FD6
:103410006666000054686520274127206F6E20747F
:1034200068652073636F7065206D65616E73204100
:10343000565220436C6F636B204D6173746572202C
:103440004D6F646500004D616B652054696D6520AA
:10345000676F2066617374004D616B652054696D00
:103460006520676F206E6F726D616C004D616B65DA
:103470002054696D6520676F206261636B004D6148
:103480006B652054696D6520676F206261636B20F6
:10349000666173742100566572626F7365206F7583
:1034A00074707574206973206F6E65206F66207963
:1034B0006F7572206F7074696F6E73005468652049
:1034C000626C696E6B696E67204220776F756C6401
:1034D00020696E6469636174652061206C6F772078
:1034E000525443206261636B75702062617474652D
:1034F00072792C20627574206E6F7720697427733F
:10350000206A75737420612064656D6F00005468D3
:10351000697320626C696E6B696E67205020696EFA
:10352000646963617465732074686174207468658C
:10353000203120505053207369676E616C2069738D
:10354000206D697373696E672E20416761696E2C07
:10355000206A75737420612064656D6F000057697F
:103560006C6C20746869732067657420796F75725C
:1035700020617474656E74696F6E3F004275726E7F
:1035800020696E2070726576656E74696F6E206D4D
:103590006F7665732074686520646973706C6179F7
:1035A00020612074696E79206269742C206E6F72BC
:1035B0006D616C6C792065766572792035206D6956
:1035C0006E75746573206275742068657265206518
:1035D00076657279207365636F6E64005765206845
:1035E0006F706520796F7520656E6A6F79656420EC
:1035F000746869732064656D6F2E205468616E6B0A
:1036000020796F7520666F72207573696E672074FC
:1036100068697320447574636874726F6E6978208A
:10362000436C6F636B001BA114601BA3F8940E9492
:10363000CA000E94F2000E94860178940895F3DF88
:10364000E0E0F8E350E040E06DEF73E280E05B988B
:103650005C98460F571FE81F1491012F1F7018B96F
:10366000029505B9F6CF0F930091C00005FFFCCF7E
:103670000F910093C60008958F930F9302950F70DA
:10368000802F0E94040C082FEEDF0F910F70802F07
:103690000E94040C082FE7DF8F91089506E40E9432
:1036A000331B00270E943C1B082F0E943C1B072F46
:1036B0000E943C1B062F0E943C1B0DE00E94331B06
:1036C0000AE00E94331B08956F5F7F1D8F1D0895D0
:1036D0006C597F1D8F1D089504E6FADF0A95E9F7FE
:1036E000089561507F098F09089564567F098F09F5
:1036F000089504E6FADF0A95E9F708950091C600F7
:103700000E94331B0B3211F4DFDF32C0053711F496
:10371000DFDF2EC0053511F4DFDF2AC00D3211F4D2
:10372000E0DF26C0043611F4E0DF22C0043411F4D7
:10373000E0DF1EC00F3309F41BC0013319F4E0E0D1
:10374000F8E316C0023319F4E0E0F9E311C00333E3
:1037500019F4E0E0FAE30CC0043319F4E0E0FBE311
:1037600007C0013729F40BA10B7F0BA30E94C201F4
:0A37700095DF0F910FBF0F91189520
:10380000808386898C8F9295989C9FA2A5A8ABAE49
:10381000B0B3B6B9BCBFC1C4C7C9CCCED1D3D5D85B
:10382000DADCDEE0E2E4E6E8EAECEDEFF0F2F3F514
:10383000F6F7F8F9FAFBFCFCFDFEFEFFFFFFFFFFC9
:10384000FFFFFFFFFFFFFEFEFDFCFCFBFAF9F8F7B0
:10385000F6F5F3F2F0EFEDECEAE8E6E4E2E0DEDCC8
:10386000DAD8D5D3D1CECCC9C7C4C1BFBCB9B6B3E1
:10387000B0AEABA8A5A29F9C9895928F8C898683A9
:10388000807C797673706D6A6763605D5A575451B6
:103890004F4C494643403E3B383633312E2C2A2785
:1038A0002523211F1D1B1917151312100F0D0C0AAC
:1038B00009080706050403030201010000000000D7
:1038C00000000000000001010203030405060708D0
:1038D000090A0C0D0F1012131517191B1D1F212398
:1038E00025272A2C2E313336383B3E404346494C5F
:1038F0004F5154575A5D6063676A6D707376797C77
:10390000000102030405060708090A0B0C0D0E0F3F
:10391000101112131415161718191A1B1C1D1E1F2F
:10392000202122232425262728292A2B2C2D2E2F1F
:10393000303132333435363738393A3B3C3D3E3F0F
:10394000404142434445464748494A4B4C4D4E4FFF
:10395000505152535455565758595A5B5C5D5E5FEF
:10396000606162636465666768696A6B6C6D6E6FDF
:10397000707172737475767778797A7B7C7D7E7FCF
:10398000808182838485868788898A8B8C8D8E8FBF
:10399000909192939495969798999A9B9C9D9E9FAF
:1039A000A0A1A2A3A4A5A6A7A8A9AAABACADAEAF9F
:1039B000B0B1B2B3B4B5B6B7B8B9BABBBCBDBEBF8F
:1039C000C0C1C2C3C4C5C6C7C8C9CACBCCCDCECF7F
:1039D000D0D1D2D3D4D5D6D7D8D9DADBDCDDDEDF6F
:1039E000E0E1E2E3E4E5E6E7E8E9EAEBECEDEEEF5F
:1039F000F0F1F2F3F4F5F6F7F8F9FAFBFCFDFEFF4F
:103A000000020406080A0C0E10121416181A1C1EC6
:103A100020222426282A2C2E30323436383A3C3EB6
:103A200040424446484A4C4E50525456585A5C5EA6
:103A300060626466686A6C6E70727476787A7C7E96
:103A400080828486888A8C8E90929496989A9C9E86
:103A5000A0A2A4A6A8AAACAEB0B2B4B6B8BABCBE76
:103A6000C0C2C4C6C8CACCCED0D2D4D6D8DADCDE66
:103A7000E0E2E4E6E8EAECEEF0F2F4F6F8FAFCFE56
:103A8000FFFDFBF9F7F5F3F1EFEFEBE9E7E5E3E134
:103A9000DFDDDBD9D7D5D3D1CFCFCBC9C7C5C3C124
:103AA000BFBDBBB9B7B5B3B1AFAFABA9A7A5A3A114
:103AB0009F9D9B99979593918F8F8B898785838104
:103AC0007F7D7B79777573716F6F6B6967656361F4
:103AD0005F5D5B59575553514F4F4B4947454341E4
:103AE0003F3D3B39373533312F2F2B2927252321D4
:103AF0001F1D1B19171513110F0F0B0907050301C4
:103B000000000000000000000000000000000000B5
:103B100000000000000000000000000000000000A5
:103B20000000000000000000000000000000000095
:103B30000000000000000000000000000000000085
:103B40000000000000000000000000000000000075
:103B50000000000000000000000000000000000065
:103B60000000000000000000000000000000000055
:103B70000000000000000000000000000000000045
:103B8000FFFFFFFFFFFFFFFFFFFFFFFFFFFFFFFF45
:103B9000FFFFFFFFFFFFFFFFFFFFFFFFFFFFFFFF35
:103BA000FFFFFFFFFFFFFFFFFFFFFFFFFFFFFFFF25
:103BB000FFFFFFFFFFFFFFFFFFFFFFFFFFFFFFFF15
:103BC000FFFFFFFFFFFFFFFFFFFFFFFFFFFFFFFF05
:103BD000FFFFFFFFFFFFFFFFFFFFFFFFFFFFFFFFF5
:103BE000FFFFFFFFFFFFFFFFFFFFFFFFFFFFFFFFE5
:103BF000FFFFFFFFFFFFFFFFFFFFFFFFFFFFFFFFD5
:00000001FF
